:020000040000FA
:0400000060283C3008
:08000800A000030EA100831209
:1000100005191028831601178312B2308100422877
:100020008316011383120B191C28AE17280A031913
:100030002E17AE192D283B28AE13AE192A282E1FD5
:100040003B28AE1A3B28A701A601A501A801AE01D5
:10005000AE164228F030AE0542282D152E13AE12F2
:100060002708AB002608AA002508A9002808AC002C
:10007000F030AE0542282E0DA80DA50DA60DA70D3A
:10008000AE1AAE0A8B100B11210E8300A00E200EAB
:02009000090065
:1000C000203084008001840A80300402031C6228EE
:1000D000DB2183160C30850587018312850187019A
:1000E0000730990000309A00103083168E0083127A
:1000F000603083168F0083120030831691009F00BA
:100100008312C83083168100831231309000003092
:1001100083168C00831210308B004C2281018E01DB
:100120008F010B118B100B108C018B17B1202D1927
:10013000B320AD21B30BA428031085190314BA0D05
:10014000F0303A02031924210C1C96280C10C00B25
:1001500096284108C00085013F3083168500831230
:10016000962864000800A91F2D11A91F0800291B4B
:100170002D11291B08002B082A0629062C02031D15
:100180002D11031D08002D110130B7008B132030F5
:10019000370783169B001C141A088312A400103022
:1001A000370783169B001C141A088312A300003023
:1001B000370783169B001C141A088312A2008B17A2
:1001C00024082B02031D1E2923082A02031D1E29B1
:1001D00022082906F039A91EE039031D1E2922082C
:1001E00029050F390319062901303702031DFD289F
:1001F0003E18FD283E14AD17FE2102303702031DC4
:100200000629BE180629BE14AD170A22290922059F
:100210000F3903191E2901303702031D14293E1C12
:1002200014293E10AD17162202303702031D1D2976
:10023000BE1C1D29BE10AD1722221E29B70A03308D
:10024000370203180800C628B601B301FA30B4001B
:100250000130B5000130B70085018701AD1397214A
:100260003E22B120B30B5729031085190314BA0D90
:10027000F0303A0203198629B41F8501B41F8701A3
:10028000B40B5729B50B57290230B500013037029E
:100290000319342202303702031939223708B6080D
:1002A0000319B60003195529B603FA30B4002D1D01
:1002B00031292D11A91F3129291B3129A91E2912E4
:1002C0000F30290503193129B9012918B90AA918CC
:1002D000B90A2919B90AA919B90AB9183129391954
:1002E00031298B1320303707BC002B08BB00BB2102
:1002F00010303707BC002A08BB00BB21003037078D
:10030000BC002908BB00BB218B1791214522850128
:100310008701B70AB60103303702031C31294C228A
:1003200008000230370203190800850187011430E4
:10033000B900B1202D1D99292D11290A0319A429CD
:10034000A91F9929291B99290F302905031D9729D0
:10035000B90B9929850187010800AD1F0800AD136D
:100360001030BC003E08BB00BB213030BC003F0851
:10037000BB00BB2108003C088B1383169B001C1498
:100380001A0883128B173B02031908008B133B08D2
:1003900083161C159A0083123C0883169B00553067
:1003A0009D00AA309D009C1464009C18D4291C1147
:1003B00083128B170800831600309B001C141A0848
:1003C0008312BD00831610309B001C141A08831280
:1003D000BE00831620309B001C141A088312C10033
:1003E0000130C11BC100C1080319C10083163030A0
:1003F0009B001C141A088312BF0008008316051006
:1004000085108312051085148E018F010C10410890
:10041000C000080083160512851283120512851686
:100420008E018F010C104108C000080083160510D2
:1004300085108312851005148E018F010C10410860
:10044000C000080083160512851283128512051656
:100450008E018F010C104108C000080085013F305B
:100460008316850083120800380903398500B80017
:100470000800380930398500B80008003C30831680
:1004800085008312B801B81408000F308316850068
:0A0490008312B801B8160800080036
:084000000800000006000200A8
:02400E00CC33B1
:1042000001008100820084008800B100B200B40087
:10421000B800A100A200FF00FF00FF00FF00FF00A8
:104220000000010001000100010001000100010087
:10423000010001000100FF00FF00FF00FF00FF0080
:10424000010000000000000000000000000000006D
:10425000000000000000FF00FF00FF00FF00FF0063
:104260000000FF00FF00FF00FF00FF00FF00FF0055
:10427000FF00FF00FF00FF00FF00FF00FF00FF0046
:10428000FF00FF00FF00FF00FF00FF00FF00FF0036
:10429000FF00FF00FF00FF00FF00FF00FF00FF0026
:1042A000FF00FF00FF00FF00FF00FF00FF00FF0016
:1042B000FF00FF00FF00FF00FF00FF00FF00FF0006
:1042C000FF00FF00FF00FF00FF00FF00FF00FF00F6
:1042D000FF00FF00FF00FF00FF00FF00FF00FF00E6
:1042E000FF00FF00FF00FF00FF00FF00FF00FF00D6
:1042F000FF00FF00FF00FF00FF00FF00FF00DD00E8
:00000001FF
